:100000000C943E001895000018950000189500000B
:10001000189500001895000018950000189500002C
:10002000189500001895000018950000189500001C
:10003000189500001895000018950000189500000C
:1000400018950000189500000C94252318950000C1
:1000500018950000189500001895000018950000EC
:1000600018950000189500001895000018950000DC
:100070001895000018950000189500008FEF8DBFAF
:10008000C8EDE0EC4E2E80E18EBFD0E1F0E15F2EB6
:10009000A89584B7082E877F84BF88E1992780932D
:1000A000600090936000EEEFFFE0A0E0B1E08827F1
:1000B0008D933197E9F70E94602566248CE00E94B9
:1000C000AE25EEEDF0E080E40E94AE2558E0C89544
:1000D000802D0E94A82531965A95C9F704C01F1F8C
:1000E0001F1F20202020E2E0F1E088E40E94AE25DE
:1000F00058E0C895802D0E94A82531965A95C9F7D9
:1001000004C0202020201F1F1F1FE6E2F1E080E531
:100110000E94AE2558E0C895802D0E94A8253196F2
:100120005A95C9F704C01F1F1F1F1F1F1F1FEAE496
:10013000F1E088E50E94AE2558E0C895802D0E9428
:10014000A82531965A95C9F704C00609090620204A
:100150002020EEE6F1E080E60E94AE2558E0C8954A
:10016000802D0E94A82531965A95C9F704C0020433
:100170000E010F110F20E2E9F1E088E60E94AE25A2
:1001800058E0C895802D0E94A82531965A95C9F748
:1001900004C00A200E1111110E20E6EBF1E080E7F9
:1001A0000E94AE2558E0C895802D0E94A825319662
:1001B0005A95C9F704C008040E111F100E20EAED6D
:1001C000F1E088E70E94AE2558E0C895802D0E9496
:1001D000A82531965A95C9F704C00A2011111111AA
:1001E0000E2085E085BD80E084BD3F983E983D9817
:1001F0003C983A98209A219A239A509A519A529A66
:10020000539A549A569A3B9A089A099A559A81ECAD
:100210008093800081E08093810088E290E0A2E0FA
:10022000B1E08D939C938CE390E0A0E0B1E08D93DE
:100230009C938AE0809304010091040148E0049FAC
:10024000A5E0B1E00C92A0E0B1E00D911C914AE96B
:1002500050E0040F151F802F912F909389008093F9
:100260008800479A469A459A449A70917B017F7D0F
:1002700070937B0180E08093E60170917B017F7B2E
:1002800070937B0180E08093F30181E08093DA0139
:1002900080E0809349018CE080934A0181E0809363
:1002A0004B018CE080934C0182E080934D0180E013
:1002B00080934E0180E080934F0180E08093500155
:1002C00081E08093DC0181E08093E70170917B0104
:1002D000777F70937B0181E0809381010E944525A7
:1002E0008FE711E00E945425E8E7F6E50E943E25DD
:1002F0008FEB11E00E945425E4E8F6E50E943E25CC
:1003000085E00E94A825E8E8F6E50E943E2586E003
:100310000E94A825ECE8F6E50E943E2581E0809346
:100320007C0100917C01083518F011F00C94FD015E
:10033000ACE7B1E0EC91FF27ACE7B1E0AD90BB24B6
:10034000A1E8B1E0AA0DBB1D91E00E94512AACE7E3
:10035000B1E0AD90BB24A1E8B1E0AA0DBB1D0C91AA
:100360000F3F11F00C94BE0180E0ACE7B1E0AD901E
:10037000BB24A1E8B1E0AA0DBB1D8C9300917C01C8
:1003800048E00E94582AA4EEB1E08C930091E40169
:10039000003011F00C94D60180E0ACE7B1E0AD90F4
:1003A000BB24A1E8B1E0AA0DBB1D8C9300917C0198
:1003B00044E00E94582AAFEDB1E00C930091DF01B8
:1003C000003018F011F00C94E7010C94F10183ED6A
:1003D000AFEDB1E01C910E945425E0E9F6E50E94E2
:1003E0003E2584E190E00E94F425ACE7B1E08C91D9
:1003F0008F5F8C9310F40C949101E4E6F0E0A2E09E
:10040000B1E092E00E94512AA2E0B1E00D911C916E
:100410000F3F50E0150711F00C94140288E290E0B1
:10042000A2E0B1E08D939C93E5E6F0E0A3EFB1E0AC
:1004300091E00E94512A0091F3010F3F11F00C94BA
:10044000240280E08093F301E6E6F0E0A0EFB1E063
:1004500091E00E94512A0091F0010F3F11F00C949D
:10046000340280E08093F001E7E6F0E0A6EFB1E02F
:1004700091E00E94512A0091F6010F3F11F00C9477
:10048000440280E08093F6010E94452587E0E9E27E
:100490000E947329A4E1B2E00C93E2E9F6E50E9420
:1004A0003E2586E00E94A825E6E9F6E50E943E2565
:1004B00085E00E94A825EAE9F6E50E943E2584E051
:1004C0000E94A825E0EAF6E50E943E25A8EAB0E1F0
:1004D000E4E1F2E00E94C6290E94312584EF91E018
:1004E0000E94F4250E94452500911402003018F066
:1004F00011F00C947D020C94770387E0E9E20E94EE
:10050000FE28A3E0B2E0E9E1F2E098E00E94322A9E
:1005100087E0E9E20E940329ABE0B2E0E9E1F2E022
:1005200098E00E94322A00910A02003011F00C94E7
:10053000AC0270917B01706270937B018FE711E0D8
:100540000E945425E6EAF6E50E943E2584EF91E0FC
:100550000E94F4250C94FF0287E0E3E0F2E00E94A1
:10056000682A402F00910A02041711F00C94EE0241
:100570008FE711E00E945425E8EBF6E50E943E2546
:1005800084EF91E00E94F4258FE711E00E9454254A
:10059000ECECF6E50E943E2581E080931302009189
:1005A0001302083018F011F00C94EC02A8EAB0E144
:1005B000E3E1F2E0A190BB24E2E0F2E0EA0DFB1DF2
:1005C0000E94102A0E943125A3E1B2E08C918F5F36
:1005D0008C9310F40C94CF020C94FF0270917B0169
:1005E000706270937B018FE711E00E945425E2ED69
:1005F000F6E50E943E2584EF91E00E94F42584EF09
:1006000091E00E94F4254091120200910A02041721
:1006100011F00C941E0370917B01706170937B014B
:100620008FEB11E00E945425E6EEF6E50E943E2590
:1006300084EF91E00E94F4250C94710387E0EBE0D5
:10064000F2E00E94682A402F00911202041711F074
:100650000C9460038FEB11E00E945425E8EFF6E55F
:100660000E943E2584EF91E00E94F4258FEB11E07B
:100670000E945425ECE0F7E50E943E2581E080933E
:10068000130200911302083018F011F00C945E036D
:10069000A8EAB0E1E3E1F2E0A190BB24EAE0F2E0F5
:1006A000EA0DFB1D0E94102A0E943125A3E1B2E051
:1006B0008C918F5F8C9310F40C9441030C94710314
:1006C00070917B01706170937B018FEB11E00E9450
:1006D0005425E2EDF6E50E943E2584EF91E00E946C
:1006E000F42584EF91E00E94F4250C947C03709132
:1006F0007B01706270937B01ABE7B1E08C9185FB6D
:1007000016F00C94960383ED11E00E945425E2E16B
:10071000F7E50E943E2535990C9490030C949603BE
:1007200082E390E00E94F4250C9483030E94452507
:100730008FE711E00E945425E6E2F7E50E943E258E
:1007400086E00E94A825E8E2F7E50E943E2508E041
:100750000E9439258FEB11E00E945425A8EAB0E1F0
:10076000E2E3F7E50E940D260E94312583E911E0BE
:100770000E945425E6E4F7E50E943E2583ED11E052
:100780000E945425ECE5F7E50E943E2586E00E9494
:10079000A825E0E6F7E50E943E250E947C21E1E0E5
:1007A000F0E00E9457250E948B21A8EFB1E08D91C7
:1007B0009C91ADE7B1E08D939C93A8EFB1E08D9152
:1007C0009C91AFE7B1E08D939C93E1E0F0E00E9453
:1007D000572580E08093130280E080931402789480
:1007E00070916E00716070936E000E9445250E94AA
:1007F0007C2180E080931402009114020A3018F0EA
:1008000011F00C9427040E944C180E94F11B3D9893
:10081000ABE7B1E09C9192FF04C0359B10C09B7F79
:100820009C9335990CC08AE09F9399270E94F425E8
:100830009F91359904C094609C930E942D04A4E17B
:10084000B2E08C918F5F8C9310F40C94FC030E94A7
:100850008B210C94F703F894FFCF0E94452581E08B
:1008600080937A0100917A01043018F011F00C9411
:100870003B040C943E0481E080937A013C98ABE702
:10088000B1E09C9191FF04C0349B10C09D7F9C936C
:1008900034990CC08AE09F9399270E94F4259F9178
:1008A000349904C092609C930E94AF053E98ABE7D8
:1008B000B1E09C9190FF04C0369B10C09E7F9C933A
:1008C00036990CC08AE09F9399270E94F4259F9146
:1008D000369904C091609C930E94B5053F98A1E2AF
:1008E000B2E09C9197FF04C0379B10C09F779C9308
:1008F00037990CC08AE09F9399270E94F4259F9115
:10090000379904C090689C930C94AC0500917A01CF
:10091000013011F00C94D1048FE711E00E945425AE
:10092000E0E7F7E50E943E2584E00E94A825EEE777
:10093000F7E50E943E2586E990E00E94F4253F9865
:10094000A1E2B2E09C9197FF04C0379B10C09F7753
:100950009C9337990CC08AE09F9399270E94F425B5
:100960009F91379904C090689C930C94AC053D9876
:10097000ABE7B1E09C9192FF04C0359B10C09B7F18
:100980009C9335990CC08AE09F9399270E94F42587
:100990009F91359904C094609C930E9495070C9494
:1009A000AA05023011F00C9413058FE711E00E94A4
:1009B0005425E6E8F7E50E943E2586E990E00E948E
:1009C000F4253F98A1E2B2E09C9197FF04C0379BC9
:1009D00010C09F779C9337990CC08AE09F9399270A
:1009E0000E94F4259F91379904C090689C930C94C1
:1009F000AC053D98ABE7B1E09C9192FF04C0359BFC
:100A000010C09B7F9C9335990CC08AE09F939927D7
:100A10000E94F4259F91359904C094609C930E9494
:100A2000AD160C94AA05033011F00C945C058FE709
:100A300011E00E945425EAE9F7E50E943E2584E092
:100A40000E94A825EAEAF7E50E943E2586E990E0A3
:100A50000E94F4253F98A1E2B2E09C9197FF04C068
:100A6000379B10C09F779C9337990CC08AE09F9367
:100A700099270E94F4259F91379904C090689C9310
:100A80000C94AC053D98ABE7B1E09C9192FF04C09B
:100A9000359B10C09B7F9C9335990CC08AE09F9337
:100AA00099270E94F4259F91359904C094609C93E6
:100AB0000E94440C0C94AA05043011F00C94AA0571
:100AC0008FE711E00E945425E0EBF7E50E943E25F8
:100AD00084E00E94A825EAEBF7E50E943E2584E029
:100AE0000E94A825E0ECF7E50E943E2586E990E00B
:100AF0000E94F4253F98A1E2B2E09C9197FF04C0C8
:100B0000379B10C09F779C9337990CC08AE09F93C6
:100B100099270E94F4259F91379904C090689C936F
:100B20000C94AC053D98ABE7B1E09C9192FF04C0FA
:100B3000359B10C09B7F9C9335990CC08AE09F9396
:100B400099270E94F4259F91359904C094609C9345
:100B50000E94BB050C9432040E9445250895AAE723
:100B6000B1E08C918F5F8C93089580917A018150D0
:100B700080937A0108950E94452581E080937A014F
:100B800000917A01053018F011F00C94C9050C940D
:100B9000CC0581E080937A013C98ABE7B1E09C9171
:100BA00091FF04C0349B10C09D7F9C9334990CC06E
:100BB0008AE09F9399270E94F4259F91349904C05D
:100BC00092609C930E94AF053E98ABE7B1E09C9188
:100BD00090FF04C0369B10C09E7F9C9336990CC03A
:100BE0008AE09F9399270E94F4259F91369904C02B
:100BF00091609C930E94B5053F98A1E2B2E09C9160
:100C000097FF04C0379B10C09F779C9337990CC007
:100C10008AE09F9399270E94F4259F91379904C0F9
:100C200090689C930C94940700917A01013011F024
:100C30000C9458068FE711E00E945425E6ECF7E586
:100C40000E943E2586E990E00E94F4253F98A1E2AB
:100C5000B2E09C9197FF04C0379B10C09F779C9394
:100C600037990CC08AE09F9399270E94F4259F91A1
:100C7000379904C090689C930C9494073D98ABE717
:100C8000B1E09C9192FF04C0359B10C09B7F9C9368
:100C900035990CC08AE09F9399270E94F4259F9173
:100CA000359904C094609C930E94BA120C949207E8
:100CB000023011F00C94A8068FE711E00E94542531
:100CC000EAEDF7E50E943E2584E00E94A825E8EEC3
:100CD000F7E50E943E2585E00E94A825EEEEF7E5A7
:100CE0000E943E2586E990E00E94F4253F98A1E20B
:100CF000B2E09C9197FF04C0379B10C09F779C93F4
:100D000037990CC08AE09F9399270E94F4259F9100
:100D1000379904C090689C930C9494073D98ABE776
:100D2000B1E09C9192FF04C0359B10C09B7F9C93C7
:100D300035990CC08AE09F9399270E94F4259F91D2
:100D4000359904C094609C930E9467130C94920799
:100D5000033011F00C9402078FE711E00E94542534
:100D6000E0EFF7E50E943E2585E00E94A82586E099
:100D70000E94A825EAEFF7E50E943E2586E00E9442
:100D8000A825E6E9F6E50E943E2585E00E94A82513
:100D9000EEEEF7E50E943E2586E990E00E94F425FC
:100DA0003F98A1E2B2E09C9197FF04C0379B10C02E
:100DB0009F779C9337990CC08AE09F9399270E9454
:100DC000F4259F91379904C090689C930C949407E4
:100DD0003D98ABE7B1E09C9192FF04C0359B10C0F9
:100DE0009B7F9C9335990CC08AE09F9399270E9422
:100DF000F4259F91359904C094609C930E946B14D4
:100E00000C949207043011F00C9444078FE711E022
:100E10000E945425EEEFF7E50E943E2586E990E01A
:100E20000E94F4253F98A1E2B2E09C9197FF04C094
:100E3000379B10C09F779C9337990CC08AE09F9393
:100E400099270E94F4259F91379904C090689C933C
:100E50000C9494073D98ABE7B1E09C9192FF04C0DD
:100E6000359B10C09B7F9C9335990CC08AE09F9363
:100E700099270E94F4259F91359904C094609C9312
:100E80000E9438150C949207053011F00C949207CB
:100E90008FE711E00E945425E2E1F8E50E943E252B
:100EA00085E00E94A825EAE1F8E50E943E2585E05C
:100EB0000E94A825EEE1F8E50E943E2586E990E033
:100EC0000E94F4253F98A1E2B2E09C9197FF04C0F4
:100ED000379B10C09F779C9337990CC08AE09F93F3
:100EE00099270E94F4259F91379904C090689C939C
:100EF0000C9494073D98ABE7B1E09C9192FF04C03D
:100F0000359B10C09B7F9C9335990CC08AE09F93C2
:100F100099270E94F4259F91359904C094609C9371
:100F20000E94E6150C94C005089581E080937A0133
:100F300070917B017F7770937B013D98ABE7B1E0C7
:100F40009C9192FF04C0359B10C09B7F9C93359968
:100F50000CC08AE09F9399270E94F4259F913599B0
:100F600004C094609C930E94AF053F98A1E2B2E058
:100F70009C9197FF04C0379B10C09F779C93379933
:100F80000CC08AE09F9399270E94F4259F9137997E
:100F900004C090689C930C94430C00917A0101303A
:100FA00011F00C9427088FE711E00E945425E8E225
:100FB000F8E50E943E250E946B0B83E911E00E9438
:100FC0005425AEE2B1E00E943325EAE3F8E50E9441
:100FD0003E25A7E3B1E00E94332583ED11E00E9496
:100FE0005425EEE3F8E50E943E2502E10E943925F2
:100FF00034990C941008AEE1B1E08C918F5F8C9322
:1010000000911E01073118F011F00C9409080C949E
:101010000C0880E080931E0186E990E00E94F42590
:1010200036990C94250880911E01815080931E01F1
:1010300000911E010F3F11F00C94210887E180936D
:101040001E0186E990E00E94F4250C94690B0230A1
:1010500011F00C9482088FE711E00E945425E2E41D
:10106000F8E50E943E250E946B0B83E911E00E9487
:101070005425AEE2B1E00E943325EAE3F8E50E9490
:101080003E25A7E3B1E00E94332583ED11E00E94E5
:10109000542503E00E943925EEE3F8E50E943E2541
:1010A0000FE00E94392534990C946B08ADE1B1E052
:1010B0008C918F5F8C9300911D010B3318F011F010
:1010C0000C9464080C94670880E080931D0186E905
:1010D00090E00E94F42536990C94800880911D01BF
:1010E000815080931D0100911D010F3F11F00C9460
:1010F0007C088BE380931D0186E990E00E94F42533
:101100000C94690B033011F00C94DD088FE711E0AB
:101110000E945425E6E5F8E50E943E250E946B0BEF
:1011200083E911E00E945425AEE2B1E00E9433252C
:10113000EAE3F8E50E943E25A7E3B1E00E943325EB
:1011400083ED11E00E94542506E00E943925EEE36C
:10115000F8E50E943E250CE00E94392534990C9454
:10116000C608A3E1B1E08C918F5F8C9300911301CD
:101170000B3318F011F00C94BF080C94C20880E0F7
:101180008093130186E990E00E94F42536990C942F
:10119000DB088091130181508093130100911301AA
:1011A0000F3F11F00C94D7088BE38093130186E96D
:1011B00090E00E94F4250C94690B043011F00C941B
:1011C00035098FE711E00E945425E6E6F8E50E9414
:1011D0003E250E946B0B83E911E00E945425AEE28C
:1011E000B1E00E943325EAE3F8E50E943E25A7E33B
:1011F000B1E00E94332583ED11E00E9454250AE0FE
:101200000E943925EAE7F8E50E943E2534990C94BE
:101210001E09A4E2B1E08C918F5F8C9300912401B0
:101220000E3018F011F00C9417090C941A098CE088
:101230008093240186E990E00E94F42536990C946D
:10124000330980912401815080932401009124016D
:101250000B3011F00C942F098EE08093240186E965
:1012600090E00E94F4250C94690B053011F00C9469
:101270008D098FE711E00E945425E0E8F8E50E940F
:101280003E250E946B0B83E911E00E945425AEE2DB
:10129000B1E00E943325EAE3F8E50E943E25A7E38A
:1012A000B1E00E94332583ED11E00E9454250FE048
:1012B0000E943925EEE3F8E50E943E2534990C940E
:1012C0007609A3E2B1E08C918F5F8C9300912301AA
:1012D0000C3018F011F00C946F090C94720981E035
:1012E0008093230186E990E00E94F42536990C94BE
:1012F0008B09809123018150809323010091230168
:10130000003011F00C9487098CE08093230186E96A
:1013100090E00E94F4250C94690B063011F00C94B7
:10132000E5098FE711E00E945425E4E9F8E50E9401
:101330003E250E946B0B83E911E00E945425AEE22A
:10134000B1E00E943325EAE3F8E50E943E25A7E3D9
:10135000B1E00E94332583ED11E00E94542502E1A3
:101360000E943925EEE3F8E50E943E2534990C945D
:10137000CE09A1E2B1E08C918F5F8C9300912101A5
:101380000F3118F011F00C94C7090C94CA0981E0D0
:101390008093210186E990E00E94F42536990C940F
:1013A000E309809121018150809321010091210165
:1013B000003011F00C94DF098FE18093210186E960
:1013C00090E00E94F4250C94690B073011F00C9406
:1013D000CC0A8FE711E00E945425E8EAF8E50E9464
:1013E0003E2583E911E00E9454250091220100303E
:1013F00011F00C940F0AEAEBF8E50E943E250FE08D
:101400000E94392583ED11E00E945425E0ECF8E5B7
:101410000E943E250FE00E9439250C949D0A013060
:1014200011F00C94270AE6ECF8E50E943E2500E155
:101430000E94392583ED11E00E945425EAE7F8E582
:101440000E943E2500E10E9439250C949D0A02303D
:1014500011F00C943F0AECECF8E50E943E250EE0FA
:101460000E94392583ED11E00E945425E4EDF8E552
:101470000E943E250EE00E9439250C949D0A0330FF
:1014800011F00C94570AECEDF8E50E943E250BE0B4
:101490000E94392583ED11E00E945425E6EEF8E51F
:1014A0000E943E250BE00E9439250C949D0A0430D1
:1014B00011F00C946F0AE0EFF8E50E943E250EE073
:1014C0000E94392583ED11E00E945425E4EDF8E5F2
:1014D0000E943E250EE00E9439250C949D0A05309D
:1014E00011F00C94870AE8EFF8E50E943E250DE024
:1014F0000E94392583ED11E00E945425E0E0F9E5D2
:101500000E943E250DE00E9439250C949D0A06306C
:1015100011F00C949D0AE8E0F9E50E943E250CE0EC
:101520000E94392583ED11E00E945425E2E1F9E59E
:101530000E943E250CE00E94392534990C94B50A8E
:10154000A2E2B1E08C918F5F8C9300912201063072
:1015500018F011F00C94AE0A0C94B10A80E080935C
:10156000220186E990E00E94F42536990C94CA0A7B
:1015700080912201815080932201009122010F3F2E
:1015800011F00C94C60A86E08093220186E990E06F
:101590000E94F4250C94690B083011F00C94320B66
:1015A0008FE711E00E945425ECE1F9E50E943E2509
:1015B0000BE00E94392583E911E00E94542503E0E5
:1015C0000E943925E4E2F9E50E943E2509E00E94E7
:1015D000392583ED11E00E945425ABE7B1E08C91F1
:1015E00087FB16F00C94000B03E00E943925EAE714
:1015F000F8E50E943E250FE00E9439250C940A0B65
:1016000009E00E943925EEE2F9E50E943E2508E056
:101610000E943925A6E2B0E00C9104FB81E00EF4B3
:1016200080E08F93A6E2B0E00C9106FB81E00EF41F
:1016300080E09F91892B882311F40C94300BABE749
:10164000B1E08C9187FB882780F9809580FBABE720
:10165000B1E08C9187F98C9386E990E00E94F425A3
:101660000C94690B093011F00C94690BABE7B1E0F5
:101670008C9187FB16F00C94510B0E945D190E940F
:1016800045258FEB11E00E945425E2E3F9E50E9425
:101690003E25E2E0F0E00E9457250E94F5030C94FD
:1016A000690B0E9445258FEB11E00E945425E0E470
:1016B000F9E50E943E2583E911E00E945425E0EC03
:1016C000F8E50E943E25E2E0F0E00E9457250E94E6
:1016D000F5030C949D07A0E4B1E0EEE1F1E00E9477
:1016E000C629E0E4F1E0A8EAB0E10E942C2AE8EA89
:1016F000F0E1A0E4B1E01127222702E033270E94A5
:101700000C28E0E4F1E0AEE2B1E00E942C2AAEE267
:10171000B1E00E942A25E0E5F9E50E940D26A0E44B
:10172000B1E0EDE1F1E00E94C629E0E4F1E0A8EAD1
:10173000B0E10E942C2AE8EAF0E1A0E4B1E0112730
:10174000222702E033270E940C28E0E4F1E0AEE219
:10175000B1E00E942A250E942C2AAEE2B1E00E944C
:101760002A25E0E5F9E50E940D26A0E4B1E0E3E1D9
:10177000F1E00E94C629E0E4F1E0A8EAB0E10E94AD
:101780002C2AE8EAF0E1A0E4B1E01127222702E0E8
:1017900033270E940C28E0E4F1E0AEE2B1E00E94C1
:1017A0002A250E942C2AA0E4B1E0E4E2F1E00E94A4
:1017B000C629E0E4F1E0A8EAB0E10E942C2AE8EAB8
:1017C000F0E1A0E4B1E01127222702E033270E94D4
:1017D0000C28A7E3B1E0E2E5F9E50E940D26E0E47C
:1017E000F1E0A7E3B1E00E942A250E942C2AA7E39A
:1017F000B1E00E942A25E6E5F9E50E940D26A0E465
:10180000B1E0E3E2F1E00E94C629E0E4F1E0A8EAF9
:10181000B0E10E942C2AE8EAF0E1A0E4B1E011274F
:10182000222702E033270E940C28E0E4F1E0A7E33E
:10183000B1E00E942A250E942C2AA7E3B1E00E9471
:101840002A25E6E5F9E50E940D26A0E4B1E0E1E2F3
:10185000F1E00E94C629E0E4F1E0A8EAB0E10E94CC
:101860002C2AE8EAF0E1A0E4B1E01127222702E007
:1018700033270E940C28E0E4F1E0A7E3B1E00E94E6
:101880002A250E942C2A089581E080937A01709184
:101890007B017F7770937B013D98ABE7B1E09C9132
:1018A00092FF04C0359B10C09B7F9C9335990CC060
:1018B0008AE09F9399270E94F4259F91359904C04F
:1018C00094609C930E94AF053F98A1E2B2E09C9186
:1018D00097FF04C0379B10C09F779C9337990CC02B
:1018E0008AE09F9399270E94F4259F91379904C01D
:1018F00090689C930C94B41200917A01013011F01D
:101900000C94750D8FE711E00E945425E8E5F9E588
:101910000E943E2505E00E9439250E944E120E9439
:10192000C9118FEB11E00E945425E8E6F9E50E9409
:101930003E25A8EAB0E1EAEDF1E00E94C6290E9446
:10194000312503E00E9439258FEB1BE00E945425CE
:1019500000914901003011F00C94B40CE0E7F9E576
:101960000E943E250C94B80CE8E7F9E50E943E255C
:1019700083E91BE00E94542500914F01003011F0D3
:101980000C94C80CE2E8F9E50E943E250C94200D69
:10199000ECE8F9E50E943E2500914E01003011F07F
:1019A0000C94DF0CE2E9F9E50E943E2586E00E94F6
:1019B000A825E4E9F9E50E943E250C94200D0130AC
:1019C00011F00C94E90CE8E9F9E50E943E250C942D
:1019D000200D023011F00C94F30CEEE9F9E50E94B1
:1019E0003E250C94200D033011F00C94FD0CE4EA1C
:1019F000F9E50E943E250C94200D043011F00C9462
:101A00000E0DEAEAF9E50E943E2586E00E94A8252F
:101A1000ECEAF9E50E943E250C94200D053011F00A
:101A20000C94180DE0EBF9E50E943E250C94200D76
:101A3000063011F00C94200DE6EBF9E50E943E25EE
:101A400083ED11E00E945425ECEBF9E50E943E2560
:101A5000AFE5B1E00E94332504E00E94392583ED13
:101A60001DE00E945425E0ECF9E50E943E25A8E621
:101A7000B1E00E94332583E917E00E945425E0E994
:101A8000F6E50E943E2534990C945D0DAAEDB1E077
:101A90008C918F5F8C93409104010091DA010417BF
:101AA00018F011F00C94560D0C94590D81E08093B0
:101AB000DA0186E990E00E94F42536990C94730DC2
:101AC0008091DA0181508093DA010091DA010030CF
:101AD00011F00C946F0D809104018093DA0186E976
:101AE00090E00E94F4250C94C711023011F00C9480
:101AF000EA0D8FEB11E00E94542504E10E94392584
:101B00008FE711E00E945425A8EAB0E1EAEDF1E088
:101B10000E94C6290E943125E4ECF9E50E943E2589
:101B200008E00E94392583E911E00E94542503E072
:101B30000E943925E4E2F9E50E943E2509E00E9471
:101B4000392583ED11E00E945425009149010130AF
:101B500011F00C94B70D03E00E943925EAE7F8E58F
:101B60000E943E250DE00E9439250C94C10D09E02C
:101B70000E943925EEE2F9E50E943E2508E00E9428
:101B80003925A6E2B0E00C9104FB81E00EF480E080
:101B90008F93A6E2B0E00C9106FB81E00EF480E0AA
:101BA0009F91892B882311F40C94E80D0091490131
:101BB000003011F00C94E10D81E0809349010C9408
:101BC000E40D80E08093490186E990E00E94F425CD
:101BD0000C94C711033011F00C945E0E0091490172
:101BE000003011F00C94F70D89E080937A018FE7B3
:101BF00011E00E945425A8EAB0E1EAEDF1E00E946C
:101C0000C6290E943125E2EDF9E50E943E2583E9CF
:101C100011E00E94542503E00E943925E6EEF9E523
:101C20000E943E2507E00E94392583ED11E00E94C5
:101C3000542500914F01003011F00C942B0E03E05D
:101C40000E943925EAE7F8E50E943E250DE00E9452
:101C500039250C94350E09E00E943925EAE7F8E5AC
:101C60000E943E2507E00E943925A6E2B0E00C91D3
:101C700004FB81E00EF480E08F93A6E2B0E00C91CB
:101C800006FB81E00EF480E09F91892B882311F4FC
:101C90000C945C0E00914F01003011F00C94550E25
:101CA00081E080934F010C94580E80E080934F01A7
:101CB00086E990E00E94F4250C94C711043011F0DD
:101CC0000C94D00E8FE711E00E945425A8EAB0E1F1
:101CD000EAEDF1E00E94C6290E943125E2EFF9E524
:101CE0000E943E2504E00E9439258FEB11E00E94FE
:101CF000542500914F01003011F00C94850EE2E064
:101D0000FAE50E943E250C94890EE8E0FAE50E946F
:101D10003E250E94C91183E911E00E945425AFE5D8
:101D2000B1E00E9433250FE00E94392583ED11E0D8
:101D30000E945425EEE3F8E50E943E2502E10E9450
:101D4000392534990C94B90EAAE4B1E08C918F5FD7
:101D50008C9300914A01073118F011F00C94B20EE7
:101D60000C94B50E80E080934A0186E990E00E94D1
:101D7000F42536990C94CE0E80914A0181508093BF
:101D80004A0100914A010F3F11F00C94CA0E87E1FD
:101D900080934A0186E990E00E94F4250C94C711D3
:101DA000053011F00C94420F8FE711E00E9454258A
:101DB000A8EAB0E1EAEDF1E00E94C6290E943125CF
:101DC000E2EFF9E50E943E2504E00E9439258FEB01
:101DD00011E00E94542500914F01003011F00C9445
:101DE000F70EE2E0FAE50E943E250C94FB0EE8E0D7
:101DF000FAE50E943E250E94C91183E911E00E9484
:101E00005425AFE5B1E00E94332583ED11E00E9437
:101E1000542503E00E943925EEE3F8E50E943E25B3
:101E20000FE00E94392534990C942B0FABE4B1E0FC
:101E30008C918F5F8C9300914B010B3318F011F054
:101E40000C94240F0C94270F80E080934B0186E9BB
:101E500090E00E94F42536990C94400F80914B013C
:101E6000815080934B0100914B010F3F11F00C9476
:101E70003C0F8BE380934B0186E990E00E94F425B0
:101E80000C94C711063011F00C94B40F8FE711E0D9
:101E90000E945425A8EAB0E1EAEDF1E00E94C629CB
:101EA0000E943125EEE0FAE50E943E2504E00E9402
:101EB00039258FEB11E00E94542500914F0100302D
:101EC00011F00C94690FE2E0FAE50E943E250C94B3
:101ED0006D0FE8E0FAE50E943E250E94C91183E9F2
:101EE00011E00E945425A8E6B1E00E9433250FE0DE
:101EF0000E94392583ED11E00E945425EEE3F8E5B8
:101F00000E943E2502E10E94392534990C949D0FD0
:101F1000ACE4B1E08C918F5F8C9300914C01073160
:101F200018F011F00C94960F0C94990F80E08093A8
:101F30004C0186E990E00E94F42536990C94B20F8A
:101F400080914C01815080934C0100914C010F3FD6
:101F500011F00C94AE0F87E180934C0186E990E07C
:101F60000E94F4250C94C711073011F00C94261030
:101F70008FE711E00E945425A8EAB0E1EAEDF1E014
:101F80000E94C6290E943125EEE0FAE50E943E2516
:101F900004E00E9439258FEB11E00E945425009146
:101FA0004F01003011F00C94DB0FE2E0FAE50E94E3
:101FB0003E250C94DF0FE8E0FAE50E943E250E94E2
:101FC000C91183E911E00E945425A8E6B1E00E94FE
:101FD000332583ED11E00E94542503E00E9439254A
:101FE000EEE3F8E50E943E250FE00E943925349982
:101FF0000C940F10ADE4B1E08C918F5F8C93009145
:102000004D010B3318F011F00C9408100C940B10C8
:1020100080E080934D0186E990E00E94F425369996
:102020000C94241080914D01815080934D010091BA
:102030004D010F3F11F00C9420108BE380934D0164
:1020400086E990E00E94F4250C94C711083011F045
:102050000C94211100914F01003011F00C943310B9
:1020600089E080937A018FE711E00E945425A8EA65
:10207000B0E1EAEDF1E00E94C6290E943125EEE1CF
:10208000FAE50E943E2504E00E94392583E911E02B
:102090000E94542500914E01003011F00C94641000
:1020A000EAEBF8E50E943E250FE00E94392583ED1A
:1020B00011E00E945425E0ECF8E50E943E250FE077
:1020C0000E9439250C94F210013011F00C947C1010
:1020D000E6ECF8E50E943E2500E10E94392583EDFB
:1020E00011E00E945425EAE7F8E50E943E2500E150
:1020F0000E9439250C94F210023011F00C949410C7
:10210000ECECF8E50E943E250EE00E94392583EDB7
:1021100011E00E945425E4EDF8E50E943E250EE012
:102120000E9439250C94F210033011F00C94AC107D
:10213000ECEDF8E50E943E250BE00E94392583ED89
:1021400011E00E945425E6EEF8E50E943E250BE0E2
:102150000E9439250C94F210043011F00C94C41034
:10216000E0EFF8E50E943E250EE00E94392583ED60
:1021700011E00E945425E4EDF8E50E943E250EE0B2
:102180000E9439250C94F210053011F00C94DC10EB
:10219000E8EFF8E50E943E250DE00E94392583ED29
:1021A00011E00E945425E0E0F9E50E943E250DE093
:1021B0000E9439250C94F210063011F00C94F210A4
:1021C000E8E0F9E50E943E250CE00E94392583ED08
:1021D00011E00E945425E2E1F9E50E943E250CE061
:1021E0000E94392534990C940A11AEE4B1E08C9127
:1021F0008F5F8C9300914E01063018F011F00C9413
:1022000003110C94061180E080934E0186E990E062
:102210000E94F42536990C941F1180914E01815033
:1022200080934E0100914E010F3F11F00C941B1151
:1022300086E080934E0186E990E00E94F4250C949C
:10224000C711093011F00C948E118FE711E00E9434
:102250005425EEE2FAE50E943E250CE00E94392565
:102260008FEB11E00E94542505E00E94392583E997
:1022700011E00E94542503E00E943925E4E2F9E5CB
:102280000E943E2508E00E94392583ED11E00E945E
:102290005425ABE7B1E08C9187FB16F00C945C11F0
:1022A00003E00E943925EAE7F8E50E943E250CE0AC
:1022B0000E9439250C94661109E00E943925EEE24E
:1022C000F9E50E943E2507E00E943925A6E2B0E02C
:1022D0000C9104FB81E00EF480E08F93A6E2B0E065
:1022E0000C9106FB81E00EF480E09F91892B8823FE
:1022F00011F40C948C11ABE7B1E08C9187FB88272B
:1023000080F9809580FBABE7B1E08C9187F98C93E5
:1023100086E990E00E94F4250C94C7110A3011F070
:102320000C94C711ABE7B1E08C9187FB16F00C94CD
:10233000AE110E94D8190E9445258FEB11E00E9432
:102340005425E2E3F9E50E943E25E2E0F0E00E9438
:10235000572581E080937A010C94C7110E9445258E
:102360008FEB11E00E945425E0E4F9E50E943E2540
:1023700083E911E00E945425E0ECF8E50E943E2537
:10238000E2E0F0E00E94572581E080937A010C940E
:102390004C0CA1E7B1E0EAE4F1E00E94C629E1E7D4
:1023A000F1E0A8EAB0E10E942C2AE8EAF0E1A1E716
:1023B000B1E01127222702E033270E940C28E1E731
:1023C000F1E0AFE5B1E00E942C2AAFE5B1E00E9458
:1023D0002A25E0E5F9E50E940D26A1E7B1E0EBE44E
:1023E000F1E00E94C629E1E7F1E0A8EAB0E10E942D
:1023F0002C2AE8EAF0E1A1E7B1E01127222702E068
:1024000033270E940C28E1E7F1E0AFE5B1E00E943C
:102410002A250E942C2AA1E7B1E0ECE4F1E00E9419
:10242000C629E1E7F1E0A8EAB0E10E942C2AE8EA37
:10243000F0E1A1E7B1E01127222702E033270E9453
:102440000C28E1E7F1E0A8E6B1E00E942C2AA8E61A
:10245000B1E00E942A25E0E5F9E50E940D26A1E7FA
:10246000B1E0EDE4F1E00E94C629E1E7F1E0A8EA7D
:10247000B0E10E942C2AE8EAF0E1A1E7B1E01127DF
:10248000222702E033270E940C28E1E7F1E0A8E6CA
:10249000B1E00E942A250E942C2A08950091DA01B9
:1024A00041E0041BABEDB1E00C93ABEDB1E00C915E
:1024B00048E0049F0C92ABEDB1E0AD90BB24A2E8E4
:1024C000B1E0AA0DBB1D8C9180934901ABEDB1E049
:1024D000AD90BB24A3E8B1E0AA0DBB1D8C91809305
:1024E0004A01ABEDB1E0AD90BB24A4E8B1E0AA0D88
:1024F000BB1D8C9180934B01ABEDB1E0AD90BB2443
:10250000A5E8B1E0AA0DBB1D8C9180934C01ABED09
:10251000B1E0AD90BB24A6E8B1E0AA0DBB1D8C9143
:1025200080934D01ABEDB1E0AD90BB24A7E8B1E0E5
:10253000AA0DBB1D8C9180934E01ABEDB1E0AD9027
:10254000BB24A8E8B1E0AA0DBB1D8C9180934F017C
:10255000ABEDB1E0AD90BB24A9E8B1E0AA0DBB1D85
:102560008C918093500108950E94452581E08093CD
:102570007A010895A0E0B1E08D919C91A1EFB1E0C6
:102580008D939C938FE711E00E945425E8E3FAE5D0
:102590000E943E2583E911E00E945425EEE4FAE50D
:1025A0000E943E25A8EAB0E1E0E0F1E00E94BF29E8
:1025B0000E943125EAE5FAE50E943E25A8EAB0E14D
:1025C000E1EFF1E00E94BF290E94312534990C947B
:1025D0000013A0E0B1E00E94DC24A0E0B1E00D9186
:1025E0001C91043650E015071CF011F00C94FA12FF
:1025F0000C94001380E090E0A0E0B1E08D939C93F8
:1026000036990C941813A0E0B1E00E94E324A0E0F6
:10261000B1E00D911C91003050E015070CF402C0A0
:102620000C94181384E690E0A0E0B1E08D939C93A5
:10263000A0E0B1E00D911C914AE950E0040F151F94
:10264000802F912F909389008093880086E990E0F5
:102650000E94F4253D98ABE7B1E09C9192FF04C045
:10266000359B10C09B7F9C9335990CC08AE09F934B
:1026700099270E94F4259F91359904C094609C93FA
:102680000C9464133F98A1E2B2E09C9197FF04C0C0
:10269000379B10C09F779C9337990CC08AE09F931B
:1026A00099270E94F4259F91379904C090689C93C4
:1026B0000C945C130C94C212A1EFB1E08D919C912B
:1026C000A0E0B1E08D939C930E9445250895A2E07F
:1026D000B1E08D919C91A8EEB1E08D939C938FE732
:1026E00011E00E945425EAEDF7E50E943E2584E0C2
:1026F0000E94A825EEE5FAE50E943E2583E910E058
:102700000E945425E6E6FAE50E943E2583E91AE098
:102710000E945425EAE6FAE50E943E2583E911E18C
:102720000E945425EEE6FAE50E943E258FEB11E06B
:102730000E945425E4E7FAE50E943E2584E00E94C9
:10274000A825ECE7FAE50E943E25A8EAB0E1E2E020
:10275000F1E00E94BF290E943125EAE5FAE50E94D6
:102760003E2534990C94DD13A2E0B1E00D911C914B
:102770004AE050E0040F151FA2E0B1E00D931C9356
:10278000A2E0B1E00D911C91043650E015071CF059
:1027900011F00C94CD130C94D31380E090E0A2E0E0
:1027A000B1E08D939C9383EDA7EEB1E01C910E9464
:1027B0005425EEEEF7E50E943E2536990C94071459
:1027C000A2E0B1E00D911C914AE050E0041B150B12
:1027D000A2E0B1E00D931C93A2E0B1E00D911C9139
:1027E000003050E015070CF402C00C94FD1384E691
:1027F00090E0A2E0B1E08D939C9383EDA7EEB1E071
:102800001C910E945425EEEEF7E50E943E250091B2
:10281000020145E00E94582AA7EEB1E00C93009116
:10282000E701003011F00C94181481E08093E70167
:1028300083EDA7EEB1E01C910E945425E2E8FAE591
:102840000E943E253D98ABE7B1E09C9192FF04C009
:10285000359B10C09B7F9C9335990CC08AE09F9359
:1028600099270E94F4259F91359904C094609C9308
:102870000C9460143F98A1E2B2E09C9197FF04C0D1
:10288000379B10C09F779C9337990CC08AE09F9329
:1028900099270E94F4259F91379904C090689C93D2
:1028A0000C94581486E990E00E94F4250C94961339
:1028B000A8EEB1E08D919C91A2E0B1E08D939C9344
:1028C0000E944525E4E6F0E0A2E0B1E092E07BE77B
:1028D0000E94402A08958091F0018093EF018FE7D4
:1028E00011E00E945425E0EFF7E50E943E2585E0C7
:1028F0000E94A82586E00E94A825EAEFF7E50E943D
:102900003E2586E00E94A825E6E9F6E50E943E25E0
:1029100085E00E94A825EEEEF7E50E943E258FEBAC
:1029200011E00E945425E4E8FAE50E943E2586E085
:102930000E94A825EAE8FAE50E943E2583E911E015
:102940000E94542503E00E943925E4E2F9E50E9443
:102950003E2508E00E94392583ED11E00E945425B0
:102960000091F001013011F00C94C21403E00E94B8
:102970003925EAE7F8E50E943E250CE00E9439255A
:102980000C94CC1409E00E943925EEE2F9E50E948E
:102990003E2507E00E943925A6E2B0E00C9104FB39
:1029A00081E00EF480E08F93A6E2B0E00C9106FB8C
:1029B00081E00EF480E09F91892B882311F40C9420
:1029C000F3140091F001003011F00C94EC1481E04C
:1029D0008093F0010C94EF1480E08093F00186E97D
:1029E00090E00E94F42582E390E00E94F4253D9857
:1029F000ABE7B1E09C9192FF04C0359B10C09B7F78
:102A00009C9335990CC08AE09F9399270E94F425E6
:102A10009F91359904C094609C930C942D153F9818
:102A2000A1E2B2E09C9197FF04C0379B10C09F7752
:102A30009C9337990CC08AE09F9399270E94F425B4
:102A40009F91379904C090689C930C9429150C941D
:102A5000AC148091EF018093F0010E944525E6E6D9
:102A6000F0E0A0EFB1E091E07BE70E94402A0895FA
:102A70008091F3018093F4018FE711E00E945425C7
:102A8000EEEFF7E50E943E2583E911E00E94542510
:102A900003E00E943925E2E9FAE50E943E2508E0BC
:102AA0000E94392583ED11E00E9454250091F30125
:102AB000003011F00C94681503E00E943925E4ED14
:102AC000F8E50E943E250AE00E9439250C94721513
:102AD0000BE00E943925EAE7F8E50E943E2505E073
:102AE0000E943925A6E2B0E00C9104FB81E00EF4CF
:102AF00080E08F93A6E2B0E00C9106FB81E00EF43B
:102B000080E09F91892B882311F40C949015A3EFFA
:102B1000B1E08C9180958C9386E990E00E94F42539
:102B20003D98ABE7B1E09C9192FF04C0359B10C08B
:102B30009B7F9C9335990CC08AE09F9399270E94B4
:102B4000F4259F91359904C094609C930C94C6150C
:102B50003F98A1E2B2E09C9197FF04C0379B10C060
:102B60009F779C9337990CC08AE09F9399270E9486
:102B7000F4259F91379904C090689C930C94C215DA
:102B80000C9452158091F4018093F3010091F301AC
:102B9000013011F00C94D1158BE0809304010C945A
:102BA000D4158AE0809304010091040148E0049F59
:102BB000A5E0B1E00C920E944525E5E6F0E0A3EF28
:102BC000B1E091E07BE70E94402A08958091F601F0
:102BD0008093F7018FE711E00E945425E2E1F8E5C8
:102BE0000E943E2585E00E94A825EAE1F8E50E94C2
:102BF0003E2585E00E94A825E0EAFAE50E943E25F0
:102C000083E911E00E94542501E00E943925E6EA9B
:102C1000FAE50E943E2583ED11E00E9454250091C3
:102C2000F601003011F00C94211601E00E943925C4
:102C3000E0ECF8E50E943E250EE00E9439250C9458
:102C40003F16013011F00C94311608E00E9439252E
:102C5000E0ECF8E50E943E2507E00E9439250C943F
:102C60003F16023011F00C943F160FE00E943925F8
:102C7000EAE7F8E50E943E2501E00E9439253499F3
:102C80000C945716A6EFB1E08C918F5F8C93009156
:102C9000F601023018F011F00C9450160C945316F3
:102CA00080E08093F60186E990E00E94F425369951
:102CB0000C946C168091F60181508093F60100917E
:102CC000F601003010F00C94681682E08093F60153
:102CD00086E990E00E94F4253D98ABE7B1E09C9135
:102CE00092FF04C0359B10C09B7F9C9335990CC00C
:102CF0008AE09F9399270E94F4259F91359904C0FB
:102D000094609C930C94A2163F98A1E2B2E09C912F
:102D100097FF04C0379B10C09F779C9337990CC0D6
:102D20008AE09F9399270E94F4259F91379904C0C8
:102D300090689C930C949E160C940B168091F7014E
:102D40008093F6010E944525E7E6F0E0A6EFB1E0AA
:102D500091E07BE70E94402A089581E080937A0108
:102D600070917B017F7770937B0180E08093DE011F
:102D700080E080937C0100917C010C3018F011F010
:102D80000C94EA16EAEAF9E4ACE7B1E08C919927F1
:102D9000AFEDB1E00E94EF278FEBAFEDB1E01C91FA
:102DA0000E945425ECE8F9E4ACE7B1E08C91992756
:102DB0000E94F227A0EEB1E00E940D26A0EEB1E045
:102DC0000E943325ACE7B1E08C918F5F8C9310F4B7
:102DD0000C94BB163D98ABE7B1E09C9192FF04C008
:102DE000359B10C09B7F9C9335990CC08AE09F93C4
:102DF00099270E94F4259F91359904C094609C9373
:102E00000E94BE173F98A1E2B2E09C9197FF04C0D8
:102E1000379B10C09F779C9337990CC08AE09F9393
:102E200099270E94F4259F91379904C090689C933C
:102E30000E94271800917A01013011F00C94BC1700
:102E40008FE711E00E945425E8E5F9E50E943E2550
:102E500005E00E94392583E911E00E94542504E130
:102E60000E943925EAEAF9E4AEEDB1E08C919927A8
:102E7000AFEDB1E00E94EF2783E9AFEDB1E01C9127
:102E80000E94542583E00E94A8250091DF010A30AA
:102E900011F00C945917AFEDB1E08C918F5F8C93CA
:102EA00083E9AFEDB1E01C910E94542583E00E94BC
:102EB000A8250091DF010F3011F00C946D17AFEDD4
:102EC000B1E08C918F5F8C9383E9AFEDB1E01C9101
:102ED0000E94542583E00E94A8250091DF01023161
:102EE00011F00C948F17AFEDB1E08C918F5F8C9344
:102EF00083E9AFEDB1E01C910E94542583E00E946C
:102F0000A825AFEDB1E08C918F5F8C9383E9AFED95
:102F1000B1E01C910E94542583E00E94A8253499B9
:102F20000C94A717AEEDB1E08C918F5F8C9300915C
:102F3000DE010C3018F011F00C94A0170C94A317BC
:102F400080E08093DE0186E990E00E94F4253699C6
:102F50000C94BC178091DE0181508093DE010091BA
:102F6000DE010F3F11F00C94B8178CE08093DE0166
:102F700086E990E00E94F4250C94EA160091DE01A7
:102F8000003011F00C94C81781E083B90C94261816
:102F9000013011F00C94D01782E083B90C942618FC
:102FA000023011F00C94D81788E083B90C942618DD
:102FB000033011F00C94E01781E089B90C942618C5
:102FC000043011F00C94E81782E089B90C942618AB
:102FD000053011F00C94F01784E089B90C94261890
:102FE000063011F00C94F81788E089B90C94261873
:102FF000073011F00C94001880E189B90C94261860
:10300000083011F00C94081880E489B90C94261843
:10301000093011F00C94101888E086B90C94261829
:103020000A3011F00C9418180E9436180C942618C7
:103030000B3011F00C94201881E080B90C94261804
:103040000C3011F00C94261882E080B9089528986D
:1030500029982B98589859985A985B985C985E983C
:103060004398109811980E94F503089581E083B960
:1030700082E083B988E083B981E089B982E089B9C7
:1030800084E089B988E089B980E189B980E489B9A7
:1030900088E086B9089508950E94E42A10EA0E9403
:1030A000FC2A12E00E94FC2A0E94E42A11EA0E94F3
:1030B000FC2A0E941B2BA3E1B1E01C930E941B2B56
:1030C000ADE1B1E01C930E941B2BAEE1B1E01C937B
:1030D0000E941B2BAFE1B1E01C930E94192BA0E2D0
:1030E000B1E01C930E94F32A80911F018093240178
:1030F00096E0A4E2B1E00E941B26009124010F9308
:103100008CE00E94DA25482F0F91040FA4E2B1E071
:103110000C93E894AFE1B1E08C9187F98C93E8943B
:10312000AFE1B1E08C9186F98C938091200180937E
:10313000220195E0A2E2B1E00E941B26E894A0E201
:10314000B1E08C9187F98C93E894A0E2B1E08C9186
:1031500086F98C93E894A0E2B1E08C9185F98C9388
:10316000AEE1B1E08C91AEE2B1E00E94CF25AEE2DB
:10317000B1E00E942A25E0E5F9E50E940D26ADE1C7
:10318000B1E08C91AEE2B1E00E942A250E94CF25E9
:10319000AEE2B1E00E942A25E0E5F9E50E940D26A5
:1031A000A3E1B1E08C91AEE2B1E00E942A250E9439
:1031B000CF25A7E3B1E0E2E5F9E50E940D26A4E200
:1031C000B1E08C91A7E3B1E00E942A250E94CF25AF
:1031D000A7E3B1E00E942A25E6E5F9E50E940D2665
:1031E000A0E2B1E08C91A7E3B1E00E942A250E9401
:1031F000CF25A7E3B1E00E942A25E6E5F9E50E9484
:103200000D26AFE1B1E08C91A7E3B1E00E942A2541
:103210000E94CF25A3E1B1E09C910E94E125A3E1AA
:10322000B1E08C93ADE1B1E09C910E94E125ADE16C
:10323000B1E08C93AEE1B1E09C910E94E125AEE15A
:10324000B1E08C93A4E2B1E09C910E94E125A4E25C
:10325000B1E08C93AFE1B1E09C910E94E125A1E245
:10326000B1E08C93A2E2B1E09C910E94E125A2E240
:10327000B1E08C93A0E2B1E09C910E94E125A3E231
:10328000B1E08C93AEE1B1E00D9111274CE350E039
:103290000E940326ADE5B1E00D931C93ADE5B1E0CE
:1032A0000D911C91ADE1B1E04D915527040F151F13
:1032B000ADE5B1E00D931C930895A3E1B1E08C91CD
:1032C0000E94DA25A5E2B1E08C93ADE1B1E08C91EA
:1032D0000E94DA25A6E2B1E08C93AEE1B1E08C91D8
:1032E0000E94DA25A7E2B1E08C93A4E2B1E08C91D0
:1032F0008C508C93A4E2B1E08C910E94DA25ADE26F
:10330000B1E08C9396E0ADE2B1E00E941326A1E219
:10331000B1E08C910E94DA25AAE2B1E08C93009191
:103320002D0140912A01042BA8E2B1E00C93A2E206
:10333000B1E08C910E94DA25ABE2B1E08C9395E08C
:10334000ABE2B1E00E941326A3E2B1E08C910E94AF
:10335000DA25ACE2B1E08C9300912B0140912C0175
:10336000042BA9E2B1E00C930E94E42A10EA0E9427
:10337000FC2A12E00E94FC2AA5E2B1E01C910E9406
:10338000FC2AA6E2B1E01C910E94FC2AA7E2B1E06F
:103390001C910E94FC2AA8E2B1E01C910E94FC2A28
:1033A000A9E2B1E01C910E94FC2A0E94F32A089530
:1033B0000091DA0141E0041BABEDB1E00C93ABED01
:1033C000B1E00C9148E0049F0C92ABEDB1E08C9120
:1033D0008F5F8C93ABEDB1E0EC91FF27A9E4B1E0F6
:1033E00091E07BE70E94402A80914901ABEDB1E07A
:1033F000AD90BB24A1E8B1E0AA0DBB1D8C93ABED51
:10340000B1E08C918F5F8C93ABEDB1E0EC91FF2735
:10341000AAE4B1E091E07BE70E94402A80914A0152
:10342000ABEDB1E0AD90BB24A1E8B1E0AA0DBB1DAE
:103430008C93ABEDB1E08C918F5F8C93ABEDB1E0F1
:10344000EC91FF27ABE4B1E091E07BE70E94402ADA
:1034500080914B01ABEDB1E0AD90BB24A1E8B1E0B0
:10346000AA0DBB1D8C93ABEDB1E08C918F5F8C935B
:10347000ABEDB1E0EC91FF27ACE4B1E091E07BE78C
:103480000E94402A80914C01ABEDB1E0AD90BB248D
:10349000A1E8B1E0AA0DBB1D8C93ABEDB1E08C911E
:1034A0008F5F8C93ABEDB1E0EC91FF27ADE4B1E021
:1034B00091E07BE70E94402A80914D01ABEDB1E0A5
:1034C000AD90BB24A1E8B1E0AA0DBB1D8C93ABED80
:1034D000B1E08C918F5F8C93ABEDB1E0EC91FF2765
:1034E000AEE4B1E091E07BE70E94402A80914E017A
:1034F000ABEDB1E0AD90BB24A1E8B1E0AA0DBB1DDE
:103500008C93ABEDB1E08C918F5F8C93ABEDB1E020
:10351000EC91FF27AFE4B1E091E07BE70E94402A05
:1035200080914F01ABEDB1E0AD90BB24A1E8B1E0DB
:10353000AA0DBB1D8C93ABEDB1E08C918F5F8C938A
:10354000ABEDB1E0EC91FF27A0E5B1E091E07BE7C6
:103550000E94402A80E0ABEDB1E0AD90BB24A1E831
:10356000B1E0AA0DBB1D8C93089581E08093DD012D
:1035700080E08093E50188E080937C014091050123
:1035800000917C01041718F011F00C94CD1BACE7EE
:10359000B1E0AD90BB24A1E8B1E0AA0DBB1D0C9138
:1035A000013011F00C94D91AA5EEB1E08C918F5F27
:1035B0008C930091DD01013011F00C94F01AACE70E
:1035C000B1E0AD90BB24A1E8B1E0AA0DBB1D8C9188
:1035D00080FBA5E2B0E08C9180F98C930C94C01B29
:1035E000023011F00C94051BACE7B1E0AD90BB24A8
:1035F000A1E8B1E0AA0DBB1D8C9180FBA5E2B0E073
:103600008C9181F98C930C94C01B033011F00C94B5
:103610001A1BACE7B1E0AD90BB24A1E8B1E0AA0D64
:10362000BB1D8C9180FBA5E2B0E08C9183F98C935B
:103630000C94C01B043011F00C942F1BACE7B1E0CC
:10364000AD90BB24A1E8B1E0AA0DBB1D8C9180FB1D
:10365000ABE2B0E08C9180F98C930C94C01B0530E8
:1036600011F00C94441BACE7B1E0AD90BB24A1E891
:10367000B1E0AA0DBB1D8C9180FBABE2B0E08C9158
:1036800081F98C930C94C01B063011F00C94591BDB
:10369000ACE7B1E0AD90BB24A1E8B1E0AA0DBB1D41
:1036A0008C9180FBABE2B0E08C9182F98C930C940E
:1036B000C01B073011F00C946E1BACE7B1E0AD906D
:1036C000BB24A1E8B1E0AA0DBB1D8C9180FBABE24D
:1036D000B0E08C9183F98C930C94C01B083011F0EE
:1036E0000C94831BACE7B1E0AD90BB24A1E8B1E042
:1036F000AA0DBB1D8C9180FBABE2B0E08C9184F9EC
:103700008C930C94C01B093011F00C94981BACE7FF
:10371000B1E0AD90BB24A1E8B1E0AA0DBB1D8C9136
:1037200080FBABE2B0E08C9186F98C930C94C01BCB
:103730000A3011F00C94AD1BACE7B1E0AD90BB24A6
:10374000A1E8B1E0AA0DBB1D8C9180FBA8E2B0E01E
:103750008C9183F98C930C94C01B0B3011F00C945A
:10376000C01BACE7B1E0AD90BB24A1E8B1E0AA0D6D
:10377000BB1D8C9180FBA2E2B0E08C9181F98C930F
:10378000ADEDB1E08C918F5F8C93ACE7B1E08C91A3
:10379000885F8C9310F40C94BE1A0091E501003000
:1037A00018F011F00C94D61B0C94E41B0091F3015B
:1037B000003011F00C94E11B119A8CE291E00E9410
:1037C000F425109A0C94F01B10980091F30100302E
:1037D00011F00C94F01B8CE291E00E94F4251198FA
:1037E0000895A3E1B2E08C918F5F8C930E94B51A8B
:1037F000E2E0F1E0D190E0808FEFE7FE8827F82E3D
:10380000082F0E9485260E94B726ECE6F6E50E9466
:10381000BB270E945A27EDE0F0E0AAEEB1E00E943B
:10382000312AE0E7F6E50E94C427EAEEF1E00E94C3
:1038300061260E942827EDE0F0E0AAEEB1E00E94A8
:10384000312AEAEEF1E00E942326AEEEB1E0DC92EE
:103850000091F001013081E009F080E08F93009148
:10386000E6010F3080E010F009F081E09F9189239C
:10387000882311F40C94431C70917B017064709345
:103880007B010C94481C70917B017F7B70937B01C2
:103890004091EE0100911302041718F011F00C94FE
:1038A000AC1D8FE711E00E945425AEE2B1E00E940A
:1038B0003325EAE3F8E50E943E25A7E3B1E00E9444
:1038C00033258FEB11E00E94542509E00E94392531
:1038D0008FEB1CE00E94542500912201003011F072
:1038E0000C94861CE2E9F9E50E943E2586E00E94E0
:1038F000A825EAEBFAE50E943E2585E00E94A8256E
:10390000EEEBFAE50E943E250C94E31C013011F029
:103910000C94901CE4ECFAE50E943E250C94E31C08
:10392000023011F00C949A1CEEECFAE50E943E2550
:103930000C94E31C033011F00C94B91CE8EDFAE58B
:103940000E943E2587E00E94A825ECEDFAE50E9442
:103950003E2585E00E94A825EEEDFAE50E943E2571
:1039600085E00E94A825E2EEFAE50E943E250C942F
:10397000E31C043011F00C94CA1CEAEAF9E50E9439
:103980003E2586E00E94A825E4EEFAE50E943E2549
:103990000C94E31C053011F00C94D41CECEEFAE509
:1039A0000E943E250C94E31C063011F00C94E31C9D
:1039B000E6EFFAE50E943E2584E00E94A825EAEFA2
:1039C000FAE50E943E258FEB1BE00E945425EEEEA7
:1039D000F7E50E943E2583E91BE00E945425EEEEA8
:1039E000F7E50E943E2581E08093DD0188E0809329
:1039F0007C014091050100917C01041718F011F041
:103A00000C94621D83E9ADEDB1E01C910E94542538
:103A1000ACE7B1E0AD90BB24A1E8B1E0AA0DBB1DBD
:103A20000C91013011F00C94411D0091DD010A3020
:103A300010F40C94371D0091DD014AE00E94582AD1
:103A4000A5EFB1E08C93A8EAB0E1E5EFF1E00E94C8
:103A5000C6290E9431258FEBADEDB1E01C910E948B
:103A60005425E0E0FBE50E943E250C943F1DA8EAAA
:103A7000B0E1EDEDF1E00E94C6290E9431250C94E1
:103A8000551DE2E0FBE50E943E250091DD010A3074
:103A900010F40C94551D8FEBADEDB1E01C910E941C
:103AA0005425EEEEF7E50E943E25ADEDB1E08C9198
:103AB0008F5F8C93ACE7B1E08C91885F8C9310F4AE
:103AC0000C94F91C0091F301003011F00C94711D5D
:103AD00083E91CE00E94542509E00E9439250C94DA
:103AE000781D83E91DE00E94542508E00E943925D5
:103AF00083ED1FE00E9454250091F001013011F088
:103B00000C949C1DABE7B1E08C9186FB16F00C94F5
:103B10008F1DE4E0FBE50E943E250C949A1DECE02D
:103B2000FBE50E943E2584E00E94A825E0E1FBE53C
:103B30000E943E250C949F1D06E00E9439250E949C
:103B4000EA2100911302083711F00C94AA1D80E0BD
:103B5000809313020C94221E80911E018093060113
:103B60000E94231E81E08093120180910B018093BB
:103B700011010E94681E85E080931201809110015E
:103B8000809311010E94681EA2E1B1E08C918C5FCC
:103B90008C930E94512180911D01809306010E9407
:103BA000231E8BE08093120180910B018093110101
:103BB0000E94681E8FE08093120180911001809313
:103BC00011010E94681EA4E1B1E0E3E1F1E00E946E
:103BD000C629E4E1F1E0A8EAB0E10E942C2AE8EA73
:103BE000F0E1A4E1B1E01127222702E033270E948F
:103BF0000C288FE713E10E945425A4E1B1E00E9454
:103C000033258FEB13E10E94542502E00E943925F1
:103C100083E913E10E94542502E00E94392583EDD7
:103C200013E10E94542502E00E94392500911302FD
:103C3000083718F011F00C941F1E0C94221E80E01F
:103C4000809313020895E4E7F6E50E94C427E6E0B6
:103C5000F1E0D080EE24FF2400270E9485260E94F8
:103C6000D226EDE0F0E0A7E0B1E00E94312AE7E0E3
:103C7000F1E00E94972AEDE0F0E00E942326ABE0FD
:103C8000B1E0DC92E7E0F1E00E94782AEDE0F0E0BC
:103C9000ACE0B1E00E94312AE4E7F6E50E94C427D7
:103CA000ECE0F1E00E9461260E942827EDE0F0E0C0
:103CB000ACE0B1E00E94312AECE0F1E00E94D62AAB
:103CC000EDE0F0E00E942326A0E1B1E0DC9208954F
:103CD00000911101003011F00C94B61E8FE7A2E1A3
:103CE000B1E01C910E94542582E00E94A82580E04A
:103CF0000E94A82582E00E94A82501E00E943925A3
:103D00008FEBA2E1B1E01C910E94542582E00E9459
:103D1000A82501E00E94392582E00E94A82501E043
:103D20000E94392583E9A2E1B1E01C910E9454254B
:103D300082E00E94A82501E00E94392582E00E94CD
:103D4000A82501E00E94392583EDA2E1B1E01C9194
:103D50000E94542582E00E94A82581E00E94A825A7
:103D600082E00E94A82501E00E94392500911101FE
:103D7000013011F00C94EC1E8FE7A2E1B1E01C9130
:103D80000E94542582E00E94A82503E00E94392564
:103D90008FEBA2E1B1E01C910E94542582E00E94C9
:103DA000A82503E00E94392583E9A2E1B1E01C9136
:103DB0000E94542582E00E94A82503E00E94392534
:103DC00083EDA2E1B1E01C910E94542582E00E94A3
:103DD000A82503E00E94392500911101023011F05D
:103DE0000C943A1F8FE7A2E1B1E01C910E94542588
:103DF00080E00E94A82580E00E94A82582E00E9421
:103E0000A82501E00E9439258FEBA2E1B1E01C91C9
:103E10000E94542581E00E94A82581E00E94A825E7
:103E200082E00E94A82501E00E94392583E9A2E1F1
:103E3000B1E01C910E94542582E00E94A82580E0F8
:103E40000E94A82580E00E94A82501E00E94392553
:103E500083EDA2E1B1E01C910E94542582E00E9412
:103E6000A82581E00E94A82581E00E94A82501E004
:103E70000E94392500911101033011F00C94881F24
:103E80008FE7A2E1B1E01C910E94542580E00E94DE
:103E9000A82580E00E94A82582E00E94A82501E0D4
:103EA0000E9439258FEBA2E1B1E01C910E945425BC
:103EB00081E00E94A82581E00E94A82582E00E945E
:103EC000A82501E00E94392583E9A2E1B1E01C9117
:103ED0000E94542580E00E94A82580E00E94A82529
:103EE00082E00E94A82501E00E94392583EDA2E12D
:103EF000B1E01C910E94542581E00E94A82581E038
:103F00000E94A82582E00E94A82501E00E94392590
:103F100000911101043011F00C94D31F8FE7A2E13E
:103F2000B1E01C910E94542582E00E94A82501E086
:103F30000E94392582E00E94A82501E00E943925CF
:103F40008FEBA2E1B1E01C910E94542582E00E9417
:103F5000A82581E00E94A82582E00E94A82501E012
:103F60000E94392583E9A2E1B1E01C910E94542509
:103F700080E00E94A82580E00E94A82582E00E949F
:103F8000A82501E00E94392583EDA2E1B1E01C9152
:103F90000E94542502E00E94392582E00E94A82553
:103FA00001E00E94392500911101053011F00C94B7
:103FB00021208FE7A2E1B1E01C910E94542582E00C
:103FC0000E94A82580E00E94A82580E00E94A825E4
:103FD00001E00E9439258FEBA2E1B1E01C910E9423
:103FE000542582E00E94A82581E00E94A82581E056
:103FF0000E94A82501E00E94392583E9A2E1B1E0F1
:104000001C910E94542580E00E94A82580E00E9417
:10401000A82582E00E94A82501E00E94392583EDB1
:10402000A2E1B1E01C910E94542581E00E94A825E4
:1040300081E00E94A82582E00E94A82501E00E945C
:10404000392500911101063011F00C946F208FE793
:10405000A2E1B1E01C910E94542582E00E94A825B3
:1040600080E00E94A82580E00E94A82501E00E942F
:1040700039258FEBA2E1B1E01C910E94542582E02A
:104080000E94A82581E00E94A82581E00E94A82521
:1040900001E00E94392583E9A2E1B1E01C910E9470
:1040A000542582E00E94A82580E00E94A82582E095
:1040B0000E94A82501E00E94392583EDA2E1B1E02C
:1040C0001C910E94542582E00E94A82581E00E9454
:1040D000A82582E00E94A82501E00E9439250091D0
:1040E0001101073011F00C94B4208FE7A2E1B1E088
:1040F0001C910E94542580E00E94A82580E00E9427
:10410000A82582E00E94A82501E00E9439258FEBB6
:10411000A2E1B1E01C910E94542502E00E943925E1
:1041200082E00E94A82501E00E94392583E9A2E1EE
:10413000B1E01C910E94542502E00E94392582E0E2
:104140000E94A82501E00E94392583EDA2E1B1E09B
:104150001C910E94542502E00E94392582E00E94B1
:10416000A82501E00E94392500911101083011F0C5
:104170000C9402218FE7A2E1B1E01C910E9454252A
:1041800082E00E94A82580E00E94A82582E00E948B
:10419000A82501E00E9439258FEBA2E1B1E01C9136
:1041A0000E94542582E00E94A82581E00E94A82553
:1041B00082E00E94A82501E00E94392583E9A2E15E
:1041C000B1E01C910E94542582E00E94A82580E065
:1041D0000E94A82582E00E94A82501E00E943925BE
:1041E00083EDA2E1B1E01C910E94542582E00E947F
:1041F000A82581E00E94A82582E00E94A82501E070
:104200000E94392500911101093011F00C945021C0
:104210008FE7A2E1B1E01C910E94542582E00E9448
:10422000A82580E00E94A82582E00E94A82501E040
:104230000E9439258FEBA2E1B1E01C910E94542528
:1042400082E00E94A82581E00E94A82582E00E94C9
:10425000A82501E00E94392583E9A2E1B1E01C9183
:104260000E94542580E00E94A82580E00E94A82595
:1042700082E00E94A82501E00E94392583EDA2E199
:10428000B1E01C910E94542581E00E94A82581E0A4
:104290000E94A82582E00E94A82501E00E943925FD
:1042A00008958FE7A2E1B1E01C910E94542502E03D
:1042B0000E9439258FEBA2E1B1E01C910E945425A8
:1042C00080E00E94A82501E00E94392583E9A2E14F
:1042D000B1E01C910E94542581E00E94A82501E0D4
:1042E0000E94392583EDA2E1B1E01C910E94542582
:1042F00002E00E943925089587E0E9E20E945928EA
:104300005CEC87E0E9E20E94812854E487E0E9E27E
:104310000E948128089587E0E9E20E94592887E0F9
:10432000E9E2A3E0B2E00E9486295EEB87E0E9E2E1
:104330000E94812887E0A8EFB1E0E9E222E02A9319
:104340000E94A92887E0E9E20E94592887E0E9E273
:10435000ABE0B2E00E9486295EEB87E0E9E20E94D2
:10436000812887E0A1E0B2E0E9E222E02A930E94FE
:10437000A928A8EFB1E00D911C914AE050E00E94FD
:104380000326A8EFB1E00D931C93A8EFB1E00D91C7
:104390001C9140E150E00E94F024A8EFB1E04D9361
:1043A0005C93A1E0B2E00D911C914AE050E00E94C4
:1043B0000326A1E0B2E00D931C93A1E0B2E00D91C1
:1043C0001C9140E150E00E94F024A1E0B2E04D9346
:1043D0005C930895ABE7B1E08C9185FB16F00C94EB
:1043E000FE2183ED11E00E945425E4E1FBE50E94EB
:1043F0003E2509E00E9439250C948722ADE7B1E003
:104400004D915C91A8EFB1E00D911C910417150737
:104410000CF402C00C942F22A8EFB1E00D911C9176
:10442000003050E0150781E009F480E08F93A8EF99
:10443000B1E00D911C91023553E0150781E009F4BC
:1044400080E09F918923882311F40C942F22A8EFF8
:10445000B1E08D919C91ADE7B1E08D939C93AFE776
:10446000B1E04D915C91A8EFB1E00D911C91041762
:1044700015071CF011F00C943F220C946222A8EF57
:10448000B1E00D911C91003050E0150781E009F476
:1044900080E08F93A8EFB1E00D911C91023553E0BD
:1044A000150781E009F480E09F918923882311F4A6
:1044B0000C946222A8EFB1E08D919C91AFE7B1E03E
:1044C0008D939C93AAEFB1E0E8EFF1E00E94BF2941
:1044D000EAEFF1E0A8EAB0E10E942C2AE8EAF0E174
:1044E000AAEFB1E01127222703E031E00E940C2857
:1044F00083ED11E00E945425AAEFB1E00E9433251C
:1045000083E00E94A825ECE1FBE50E943E25ABE795
:10451000B1E08C9184FB16F00C949B2283ED18E0A3
:104520000E945425E0E2FBE50E943E2509E00E943E
:1045300039250C942423ADE7B1E04D915C91A8EFAF
:10454000B1E00D911C91041715070CF402C00C94F6
:10455000CC22A8EFB1E00D911C91003050E015077E
:1045600081E009F480E08F93A8EFB1E00D911C91F8
:10457000023553E0150781E009F480E09F9189231B
:10458000882311F40C94CC22A8EFB1E08D919C917A
:10459000ADE7B1E08D939C93AFE7B1E04D915C91B5
:1045A000A8EFB1E00D911C91041715071CF011F054
:1045B0000C94DC220C94FF22A8EFB1E00D911C9129
:1045C000003050E0150781E009F480E08F93A8EFF8
:1045D000B1E00D911C91023553E0150781E009F41B
:1045E00080E09F918923882311F40C94FF22A8EF87
:1045F000B1E08D919C91AFE7B1E08D939C93AAEFD0
:10460000B1E0E1E0F2E00E94BF29EAEFF1E0A8EAC0
:10461000B0E10E942C2AE8EAF0E1AAEFB1E011270C
:10462000222703E031E00E940C2883ED18E00E946D
:104630005425AAEFB1E00E94332583E00E94A8250B
:10464000E8E2FBE50E943E2508950F921F922F920B
:104650003F924F925F927F92AF92BF920F931F93C0
:104660002F933F934F935F936F937F938F939F937A
:10467000AF93BF93CF93DF93EF93FF938FB78F9356
:10468000A1E8B1E08C918F5F8C93329B0C944B230B
:1046900080E08093E60180E08093580100918101E1
:1046A0000E3111F00C94A8240091E601043110F0B1
:1046B0000C945F23A6EEB1E08C918F5F8C93709188
:1046C0006E007E7F70936E000091DC0141E0041B60
:1046D000ABEDB1E00C93ABEDB1E00C9148E0049F81
:1046E0000C92ABEDB1E0AD90BB24A2E8B1E0AA0D15
:1046F000BB1D8C9180935101ABEDB1E0AD90BB241B
:10470000A3E8B1E0AA0DBB1D8C9180935201ABEDE3
:10471000B1E0AD90BB24A4E8B1E0AA0DBB1D8C9123
:1047200080935301ABEDB1E0AD90BB24A5E8B1E0BF
:10473000AA0DBB1D8C9180935401ABEDB1E0AD90FF
:10474000BB24A6E8B1E0AA0DBB1D8C918093550156
:10475000ABEDB1E0AD90BB24A7E8B1E0AA0DBB1D65
:104760008C9180935601ABEDB1E0AD90BB24A8E8ED
:10477000B1E0AA0DBB1D8C9180935701A2E5B1E079
:104780000D9111274CE350E00E940326A9E5B1E00A
:104790000D931C93A9E5B1E00D911C91A3E5B1E047
:1047A0004D915527040F151FA9E5B1E00D931C93FA
:1047B000A4E5B1E00D9111274CE350E00E940326DF
:1047C000ABE5B1E00D931C93ABE5B1E00D911C910D
:1047D000A5E5B1E04D915527040F151FABE5B1E0FC
:1047E0000D931C9300915101013011F00C945F2442
:1047F00000915701003011F00C942924A9E5B1E093
:104800004D915C91ADE5B1E00D911C910417150738
:1048100080E00CF081E08F93ABE5B1E04D915C91CD
:10482000ADE5B1E00D911C910417150780E00CF483
:1048300081E09F918923882311F40C94242481E042
:10484000809358010C94272480E0809358010C94A5
:104850005D24A9E5B1E04D915C91ADE5B1E00D912C
:104860001C910417150780E00CF081E08F93ABE5F5
:10487000B1E04D915C91ADE5B1E00D911C91041753
:10488000150780E00CF481E09F9189238F9340917C
:10489000220100915601041781E009F080E09F9108
:1048A0008923882311F40C945A2481E080935801C1
:1048B0000C945D2480E0809358010C94622480E085
:1048C00080935801ABE7B1E08C9186FB81E00EF05C
:1048D00080E08F930091F001013081E009F080E0E9
:1048E0009F918923882311F40C94822480E0ABEDFE
:1048F000B1E0AD90BB24A9E8B1E0AA0DBB1D8C933B
:104900000C948D2480915801ABEDB1E0AD90BB24A7
:10491000A9E8B1E0AA0DBB1D8C93ACEDB1E08C9180
:104920008F5F8C93409104010091DC01041718F013
:1049300011F00C949D240C94A02481E08093DC0160
:1049400081E08093810170916E00716070936E00C0
:104950008F918FBFFF91EF91DF91CF91BF91AF9179
:104960009F918F917F916F915F914F913F912F9187
:104970001F910F91BF90AF907F905F904F903F90AD
:104980002F901F900F901895F894FFCF31003200B0
:10499000330034003500360037003800390031303C
:1049A000002A00535A004D535A0001020304050621
:1049B0000708090A0D0F1200ED91FC91EF5FFF4F00
:1049C000FC93EE930895ED91FC91E150F040FC933F
:1049D000EE93089509D00E94032600FC10D008959C
:1049E00003D01ED001F8F9CF0024E89457FF02C08D
:1049F00009D0689400F80BD010F80124089502D073
:104A000009D00895509540954F5F5F4F0895E89401
:104A100017FF0895009510950F5F1F4F6894089534
:104A2000352F242FE894452B11F468940895512FC5
:104A3000402F0027112780E1440F551F001F111F31
:104A4000021B130B416018F4020F131F4E7F8A954F
:104A500099F708958F938D918823E9F711978F9196
:104A60000895A8EAB0E18D91882311F071D0FBCFB1
:104A7000089580E26DD00A95E1F708950E94B72766
:104A8000802D11F065D0FACF089581E067D015D060
:104A900080E864C08FE7213039F08FEB223021F0BD
:104AA00083E9233009F083ED810F0C94AE2588EE65
:104AB00093E09AD03197D9F7089583E0992794C06D
:104AC0008AEF90E00E94F4250F9A0E9A0D9A0C9AA4
:104AD0000B9A0A9A129885E090E00E94F4251398A8
:104AE00017981698159A149A139AEF93FF93ECE877
:104AF000F1E00E94E825FF91EF91139872D0139A8C
:104B0000EF93FF93ECE8F1E00E94E825FF91EF912D
:104B1000139867D0139AEF93FF93ECE8F1E00E94AB
:104B2000E825FF91EF9113985CD01498139AEF93B6
:104B3000FF93ECE8F1E00E94E825FF91EF911398D4
:104B400050D088E20BD08EE009D086E007D00895DF
:104B5000129A829505D004D044D008951298F9CFC6
:104B6000859510F4149A01C01498859510F4159A3F
:104B700001C01598859510F4169A01C01698859570
:104B800010F4179A01C01798139AEF93FF93ECE86B
:104B9000F1E00E94E825FF91EF9113980895982F76
:104BA00082958F70805D8D939F70905D9D93882717
:104BB0008C9308954AE0082F0E94582A0295802B72
:104BC0000895892F8F70905110F0865FFCCF089563
:104BD0003197F1F70895689462F80895E89462F8BF
:104BE000089581E090E000C0EF93FF93EE27E82B5B
:104BF000E92B31F0E0EAFFE03197F1F70197D1F7C7
:104C0000FF91EF9108950F92B801469F8001479F51
:104C1000100D569F100D0F9008950E94B7270D920A
:104C20000020D9F70895903029F08C91880F9A953B
:104C3000E9F78C930895903029F08C9186959A9598
:104C4000E9F78C9308953DD0992711278F2D880F70
:104C500080E8F82A802F881F08F41FEF41F08F5753
:104C6000082F07FD04C0003240F08FEF01C08827F5
:104C7000982FD82EE82EF82E09C08FE1801B082F20
:104C8000F694E794D79497950A95D1F7112351F0AC
:104C90009095D094E094F09481E0980F8827D81EE6
:104CA000E81EF81E0F2DFE2CED2CD92E0895D09461
:104CB000E094F09491E0D90E9927E91EF91E109521
:104CC0000895D190E190F190019108952191319151
:104CD000419151910895102F90E8FF0C001F092772
:104CE000990FF7941078652F90E8440F551F5927B6
:104CF000990F4795607800380895FF0C90E8902749
:104D0000110F9795F794092F0895102FBD2CDE2CC5
:104D1000EF2CF02E11234AF4B094D094E094F09448
:104D20009FEFB91AD90AE90AF90A0EE1FF2039F40E
:104D3000FE2CED2CDB2CBB240850C2F767C032F0F0
:104D40000A95BB0CDD1CEE1CFF1CF9CF0E94A926A6
:104D5000D4CFB7FE089590E8B91611F4D0FE0895A7
:104D60009FEFD91AE90AF90A09F403950895502F1B
:104D70002D2D3E2D4F2D612F08952DEC3CEC4CEC4C
:104D80005DE366270FC09DDFF2DFDD24EE2490E8AF
:104D9000F92E0FE307C09ADF05C02227332740E230
:104DA00051E46627552351F1002381F194DF71F11D
:104DB0001627005850580894050B18F407FD03C037
:104DC00025C007FD23C0469537952795F694E794AF
:104DD000D79422D0FF202AF0DD0CEE1CFF1C0150DE
:104DE00073F09D2D969548F0DD203AF4EE202AF4DC
:104DF00091E0D90E9927E91EF91E7FCF07C09FE7E2
:104E0000092FF92A9FEFD92EE92E0895DD24EE24EB
:104E1000FF240027112708959F929924AA24BB24D8
:104E200088E1D216E306F40628F0D21AE30AF40A5F
:104E3000089401C08894991CAA1CBB1CDD0CEE1CB4
:104E4000FF1C8A9571F7D92CEA2CFB2C9F900895B2
:104E500042DFE1F25038D1F216270058505808943A
:104E6000051F12F418F4CBCF08F0D0CF0BD0FF20E1
:104E70002AF0BB0CDD1CEE1CFF1C3FCF0F5F0BF4B8
:104E8000BECF3BCF9F929924AA24BB24992788E1C7
:104E9000990CAA1CBB1CDD1CEE1CFF1C30F4920EEE
:104EA000A31EB41ED91EE91EF91E8A9589F79F908C
:104EB00008950CDF10DF503829F090E869270CC006
:104EC0000AF045D01ACF5FE322273327442701C0D9
:104ED000FDDE01DF5038B1F3003899F3902F951BB8
:104EE0008BF312F434D0FACF983118F022273327FD
:104EF0004427983028F0232F342F44279850F9CF97
:104F0000992329F04695379527959A95D9F7912FAA
:104F1000962742F014D0B0F6F794E794D7940F5F39
:104F20008BF66DCF10D051F008F4C1DEFF2052F2A5
:104F3000DD0CEE1CFF1C0150CBF761CF67CFD20E0A
:104F4000E31EF41E0895D21AE30AF40A0895DF92CC
:104F5000EF92FF920F931F93D22EE32EF42E052F84
:104F6000162F6F915F914F913F912F910895C895A2
:104F7000319600200895FBDFD02CF9DFE02CF7DF1D
:104F8000F02CF5DF002D0895F2DF202DF0DF302D1D
:104F9000EEDF402DECDF502D089507FB00680EF486
:104FA0000F7757FB50680EF45F7707FD02C057FF7D
:104FB00005C0D216E306F406050708952D153E0533
:104FC0004F055007089591E005C092E003C094E0BA
:104FD00001C098E0CCDF0D929A95E1F70895E80FB3
:104FE000F91FF1CF882311F4992329F00E94B727E4
:104FF000E9F70197D9F7089591E0882321F0889483
:10500000991F8A95E9F7892F90950895883018F0AF
:1050100011968850FBCF08952E2E3F2E992781910F
:105020008D3209F093958823D1F79A95E22DF32DCF
:10503000112361F0091718F011F0101B01C0191BA2
:1050400028F021F080E28D931A95E9F780818D3266
:1050500019F48D93319604C0222311F08BE28D93C5
:10506000091738F031F0091B21F080E38D930A9580
:10507000E9F781918D938823E1F7332351F0EA2FEB
:10508000FB2F319633958E9182933A95E1F78EE21C
:105090008C9308950181082B0183128119231283B7
:1050A000EF93FF93E4E1F0E00E94E825FF91EF9198
:1050B00008950E94EE25FF270E94FC27EBDFEF9367
:1050C000FF93ECE7F7E00E94E825FF91EF91182BA2
:1050D000128309230183EF93FF93E4E1F1E00E943F
:1050E000E825FF91EF911081182311F00E94EB2524
:1050F000EF93FF93E4E6F6E00E94E825FF91EF913D
:1051000008950E94FC27FF2721E048E006C00E9486
:10511000FC27FF2729915D9148E0BCDF579510F4EB
:10512000182B1283EF93FF93E4EDF0E00E94E82543
:10513000FF91EF91182B1283EF93FF93E4E2F0E0DD
:105140000E94E825FF91EF914A9539F72A9519F7C2
:1051500008950E94FC27FF27299148E055279ADFF0
:1051600009230183EF93FF93E0E2F0E00E94E8253A
:10517000FF91EF9188941081182309F008945795B6
:10518000EF93FF93E8EDF0E00E94E825FF91EF91A7
:105190004A9529F75D932A9501F708957BDF092346
:1051A0000183EF93FF93E0E2F0E00E94E825FF9196
:1051B000EF91E8941081182309F06894EF93FF931E
:1051C000E8EDF0E00E94E825FF91EF91089562DF9D
:1051D00016F4182B1283EF93FF93E4EDF0E00E9496
:1051E000E825FF91EF91182B1283EF93FF93E4E2F0
:1051F000F0E00E94E825FF91EF9108953327309366
:1052000018023093150255DF0EF458C03091150284
:1052100030FD54C0662760931702639560931602B1
:1052200021E050EF48E079DFB9DF31F9B7DF32F93B
:10523000632F6670663009F441C0603019F031FBAD
:1052400040D025C060911602709118026717B1F026
:10525000C0F48F939F93862F8A95A9E1B2E0D6DEA2
:10526000CBDE7C9178236894772329F4E8946091CD
:105270001602609317029F918F9109C0689421D004
:1052800006C0E8941ED060911602609317029FDF5B
:1052900060911602639560931602613409F0C4CFE1
:1052A00060911702609318026623E89409F46894E9
:1052B00030F930931502E89462F80895689462F822
:1052C00008958F939F93A9E1B2E0809116028A9589
:1052D0009DDE92DE7C9116F4782B01C079237C93BD
:1052E0009F918F9108958F9389DF8F91A0E0B0E017
:1052F00056F011968F93AF93BF9385DFBF91AF9117
:105300008F910EF0F6CF0A2F1B2F0895AF93BF9306
:10531000EF93FF9338E0E9E1F2E00D9101933A95C4
:10532000E1F7FF91EF9130E4309318023327309387
:10533000150269DF38E0BF91AF91E9E1F2E00D912C
:105340004191041719F43A95D1F708950E94EB257D
:105350000895000F111F221F331F08950095109507
:10536000209530950F5F1F4F2F4F3F4F08950191AC
:1053700010810EC001911191219130810BC00191DA
:10538000108117FF05C03FEF2FEF04C000811127E8
:105390002227332737FF03C0E1DF8DE28D93CF93C0
:1053A000DF93CF92DF92EF92AA24BB24CC24DD249A
:1053B000EE2440E2CAE0DD2755E093E38881890FBF
:1053C00087FD9F7083FD907F891B89935A95A9F76C
:1053D000C0DFAA1CBB1CCC1CDD1CEE1C4A9551F77F
:1053E000E894EFE0FF2782910ED0EB30E0F71EF05B
:1053F00068948A2D0CD088278D93EF90DF90CF9002
:10540000DF91CF910895982F829501D0892F8F70C9
:10541000805D26F0803309F4089568948D93089593
:1054200041E003C042E001C044E0E40F8827F81FD8
:105430008291982F829506D0892F04D04A95C1F782
:105440000C94292A8F708A3008F0895F805D8D93D3
:10545000089588278D93089581918D938823E1F78E
:10546000089594E081918D939A95E1F70895F999C3
:10547000FECFE1BDF2BD3196089591E001C092E00A
:105480007B3751F47FB7F894F2DF8D9180BDFA9AA3
:10549000F99A9A95C9F77FBF7727089591E001C0DF
:1054A00092E0E5DFF89A80B58D939A95D1F708954B
:1054B000FF93881BF9E0001FFA9511F4FF910895FE
:1054C000881F841B18F4840F8894F5CF0894F3CFB9
:1054D00000276CE8719198E00695779577FF18F4AE
:1054E00077FD08F006279A95B9F78A9599F70895F8
:1054F000E8DBF1DB0395AAF087E1DD0CEE1CFF1C75
:105500008A9589F00A95CAF7FF205AF000240D28E1
:105510000E280F28002039F00A95DD0CEE1CFF1C28
:10552000DAF70A95EACB72CCCCDB80E003C0C9DBAA
:10553000802F8078882321F0DF92EF92FF920F93E3
:105540008F93C9DB802F839512F460DC1BC080959C
:105550008A95885E0AF415C088501AF40CD0D922B6
:1055600010C0DD2488501AF406D0E9220AC0EE24C7
:1055700002D0F92206C09FEF8770990F8A95EAF74B
:105580000895BBDB8F918823D9F35F914F913F91B1
:105590002F910F9302DD0F9199F390F302D0506891
:1055A00098CC5FE340E83327222708958ADB0F93E6
:1055B0000F7789DCBDDF8F918078082B08954198A3
:1055C0004098399838980895389A399803D038987F
:1055D00001D0399AEF93FF93E0E1F0E00E94E825D3
:1055E000FF91EF910895389A399AF4DF3898309BFB
:1055F000FECFF0DF3998EECF0894111F01C0110FD4
:1056000069F0389A18F40000399802C0399A00C03D
:10561000E1DF3898309BFECFDDDFF1CF389A399843
:10562000D9DF3898309BFECFE8943199689462F8BE
:10563000D1CF089401C08894331F11E0389A39986B
:10564000C9DF3898309BFECFC5DF88943199089424
:10565000111FA0F7389A379510F4399801C0399A7C
:10566000B9DF3898309BFECFB5DF08950000C842FF
:105670009A99993F000020415A6F6E6120616461E0
:10568000746F6B00626574006C74000073650000D9
:105690003D0045727A006B656C006B20737A0000E8
:1056A0006D613A2000004E4F2053454E534F52201B
:1056B000312020202020000053454E534F522031EE
:1056C00020435243204F4B202020200049443120CA
:1056D00000004552524F52204441544120312D5731
:1056E0004952452020004E4F2053454E534F5220E3
:1056F000322020202020000053454E534F522032AC
:1057000020435243204F4B20202020004944322088
:1057100000004552524F5221205332202D20544F29
:105720005641424200004B00737A69746574746597
:105730003A0031342D30332D323031342032323A88
:1057400033393A33340053545249435A2052414A70
:105750004D554E4420532E522E200000435A000037
:10576000482056494B544F5220432E562E200000BD
:105770004D454E55203E20525443206265006C6CCE
:1057800069742E2000004D454E55203E205A6F6E04
:1057900061207465737A742020004D454E55203E7B
:1057A000205A6F6E6120626500006C6C69742E0077
:1057B0004D454E55203E204265006C6C69740000DA
:1057C000736F6B2020004F5054203E204C434420E8
:1057D0006B6F6E747261737A74004F5054203E2068
:1057E0004E616779737A00006D20696400002000C3
:1057F0004F5054203E2045730000727A00004F50F5
:1058000054203E204D617374657220737A656C6517
:1058100070004F5054203E20420076697400207082
:105820006F727420202000004D454E55203E204FC1
:105830005241204245414C4C0000202000003D3D9B
:1058400000004D454E55203E2050455243204245D4
:10585000414C4C2000004D454E55203E204D5020DF
:105860004245414C4C004D454E55203E204556206A
:105870004245414C4C20202020003D3D3D3D000054
:105880004D454E55203E20484F4E41502042454107
:105890004C4C00004D454E55203E204E415020427C
:1058A00045414C4C202000004D454E55203E20489F
:1058B0004554204E41504A414900484554464F0006
:1058C0003D3D3D3D3D004B4544440000535A45524B
:1058D000444100003D3D3D3D3D3D00004353555496
:1058E0004F52544F4B003D3D3D3D3D3D3D3D3D0004
:1058F00050454E54454B0000535A4F4D42415400C1
:105900003D3D3D3D3D3D3D0056415341524E415090
:1059100000003D3D3D3D3D3D3D3D00004D454E546B
:1059200053453F004947454E20204E454D003D3DE3
:105930003D002020454C4D454E545645202000004A
:105940004E494E435320454C4D454E54564520003C
:105950003A00323000002E005A4F4E412056414C42
:1059600041535A5441533A005A6F6E613A20000035
:10597000496E616B74697600416B746976202020F2
:1059800000004E6170692020202020004865746965
:1059900028004800742900004B6564290000537AF0
:1059A0006529000043737529000050006E2900002E
:1059B000537A6F29000056617329000042653A004E
:1059C0004B693A00205A4F4E4120414B5449563FB3
:1059D00000002E205A4F4E41204759414B4F52490B
:1059E000534147413F004E415049202048455449CA
:1059F00000002E205A6F6E612062656B61706373C8
:105A00002E004E61706900004865746900002E2008
:105A10005A6F6E61206B696B617063732E002E206C
:105A20006D656C79696B206E61706F6E3F004D45DE
:105A30004E5453454D3F00004F5054203E204B6F75
:105A40006E747261737A74202020202000004B6FE6
:105A50006E7472617374203D2000252020006D203B
:105A60002020202000002030250035302500313056
:105A7000302500004E616779737A00006D203D206B
:105A800000002A00456E676564006C79657A76656A
:105A90003F00537A656C657020205A6F6E6100007C
:105AA00020706F7274004E696E637320202B5A6FE2
:105AB0006E6120204574682E00007466000020206E
:105AC000202000004B656464202020202000537AB1
:105AD00065726461202020004373000074007274BA
:105AE00000006B006E74656B20202000537A6F6D90
:105AF00062617420200056617300726E6170200034
:105B000031002D004E65647665730000537A000005
:105B100072617A0054312E457272000043200000F9
:0A5B200054322E457272000043005B
:00000001FF
